S01A000064656D6F70726F675F73746D3332663035312E7372656399
S31508002000880500201D350008332800083F290008E8
S3150800201000000000000000000000000000000000B2
S31508002020000000000000000000000000432900082E
S315080020300000000000000000832E00087B33000823
S3150800204087330008FB340008073500087D3500088B
S315080020507F35000881350008833500088535000876
S3150800206087350008893500088B3500088D35000846
S315080020708F35000891350008933500089535000816
S315080020809735000899350008000000009B350008C0
S315080020909D3500089F350008A1350008A3350008BE
S315080020A0A5350008A7350008A9350008AB3500088E
S315080020B0AD35000800000000AF350008000000003C
S315080020C0EE11AA55F8B50400002738002078C00795
S315080020D063D50C20AA490A680240042A06D00A6871
S315080020E0104008280BD10868C00308D5A548006821
S315080020F0800352D5606800284FD10120F1E160685D
S31508002100012806D19F480168802252020A430260CC
S3150800211024E06068002809D19A4801689A4A0A406A
S3150800212002600168994A0A40026017E0606805285B
S315080021300BD1944801688022D2020A4302600168E2
S31508002140802252020A43026008E08E4801688E4ADD
S315080021500A40026001688D4A0A40026060680028E9
S315080021600DD000F0DDFA050086480068800314D417
S3150800217000F0D6FA401B6528F6D30320B1E100F03B
S31508002180CFFA05007F480068800306D500F0C8FA34
S31508002190401B6528F6D30320A3E1207880071CD5C9
S315080021A00C2077490A680240002A06D00A681040BF
S315080021B008282AD10868C00327D472480168890705
S315080021C004D5E168012901D001208AE10168F822D5
S315080021D091432269D2000A4302602078000755D548
S315080021E0E069002840D0BF4D2868012101432960D5
S315080021F000F096FA06002868800747D400F090FA9F
S31508002200801B0328F7D303206BE1E068002819D068
S315080022105C4D286801210143296000F081FA060017
S315080022202868800706D400F07BFA801B0328F7D3BA
S31508002230032056E12868F82188432169C90001432B
S315080022402960CAE74F4D286801218843286000F0B5
S3150800225067FA060028688007BFD500F061FA801B78
S315080022600328F7D303203CE19E4D286801218843C3
S31508002270286000F055FA06002868800706D500F0A1
S315080022804FFA801B0328F7D303202AE10425206888
S315080022902840002800D183E03E008020400592496E
S315080022A009680140002908D18F490A6802430A6073
S315080022B0096808400090009801268C4F3868C005C8
S315080022C012D43868802149000143396000F028FAA1
S315080022D000903868C00507D400F022FA0099401A21
S315080022E06528F6D30320FCE0A068012805D18048BC
S315080022F0016801220A43026021E0A068002809D18A
S315080023007B480168012291430160016804229143D8
S31508002310016014E0A068052808D1754801682943BA
S315080023200160016801220A43026008E070480168FA
S315080023300122914301600168042291430160A0686B
S3150800234000280ED000F0ECF90700694800688007FD
S315080023501ED400F0E5F9C01B66498842F5D3032070
S31508002360BFE000F0DDF907006148006880070FD577
S3150800237000F0D6F9C01B5F498842F5D30320B0E0C8
S315080023800410024000100240FFFFFEFFFFFFFBFFA4
S31508002390F6B2012E04D154480168AB4A0A400260DD
S315080023A02078C0061ED5606901283DD1A74E306841
S315080023B005433560306801210143316000F0B0F90A
S315080023C005003068800706D400F0AAF9401B0328E8
S315080023D0F7D3032085E03068F8218843A169C9004E
S315080023E001433160206A00287AD0994F38680C2159
S315080023F00140082972D0206A02285DD1954D2868C7
S3150800240095490140296000F08BF900908026B604B2
S315080024102868304000282DD000F082F90099401A2B
S315080024200328F3D303205CE00421C943606988428A
S315080024300BD186480268114001600168F822914371
S31508002440A269D2000A430260CCE7804E3068054391
S315080024503560306801218843306000F061F9050075
S3150800246030688007BED500F05BF9401B0328F7D318
S31508002470032036E0794801680F229143E26A0A434D
S315080024800260386893490140A06A0843616A0143BB
S3150800249039602868802149040143296000F040F921
S315080024A004002868304000281AD100F039F9001BCA
S315080024B00328F6D3032014E0664C206866490140D9
S315080024C0216000F02DF905002068800108D500F08C
S315080024D027F9401B0328F7D3032002E0012000E078
S315080024E00020F2BD241002401C100240007000407B
S315080024F02010024089130000F3B581B000210125A0
S315080025007B4E31682940029A91420CD231680122E9
S315080025109143029A0A43326031682940029A9142ED
S3150800252001D001208FE00400022021680140002923
S3150800253006D047490A68F0239A43A36813430B60F9
S3150800254021682940002952D06168012905D14148EE
S315080025500068800311D4012075E06168022905D15D
S315080025603C480068800108D401206CE039490968B4
S315080025700840002801D1012065E0354F386803215D
S31508002580884361680143396000F0CAF800906068C2
S3150800259001280DD138680C210140042927D000F004
S315080025A0BFF80099401A53498842F3D303204AE0FA
S315080025B0606802280DD138680C210140082916D018
S315080025C000F0AEF80099401A4A498842F3D303202E
S315080025D039E038680C210140002908D000F0A0F83D
S315080025E00099401A43498842F3D303202BE0029806
S315080025F03168294088420CD2306801218843029903
S3150800260001433160306805400298854201D00120B7
S3150800261019E02078400706D50D480168364A0A4071
S31508002620E1681143016000F01BF83449084A126852
S3150800263012091207120F895CC84031490860002048
S3150800264000F074F80020FEBDFFFFFFEF34100240D3
S315080026500410024000100240FFFFFFFE2C1002404B
S3150800266010B588B004A82749102200F071F868460A
S315080026702549102200F06CF800210800080008001F
S315080026800800224800680C210140042902D00829C4
S3150800269002D017E01E4C16E00F2104AA830C0B404B
S315080026A0D45C6A461B4B1B681940515CC00306D5AF
S315080026B0174800F067F8210004004C4301E016486B
S315080026C0444300E0124C200008B010BD0C480068D6
S315080026D070470000FFFFC2FF80B5FFF7F7FF0F49FD
S315080026E00A4A1268120A5207520F895CC84002BD8C
S315080026F00020024089130000FFF8FFFF5435000848
S31508002700C000002034350008443500080410024093
S3150800271000127A002C10024000093D0070350008AE
S3150800272001480068704700BF8001002010B504000A
S31508002730FFF7CCFFFA21890000F024F800F0DCF856
S31508002740002221000020C04300F0D1F8002010BD6F
S3150800275070B4103A03D378C9103A78C0FBD253073D
S3150800276001D318C918C001D508C908C0D20704D3AF
S315080027700B880380891C801C002A01D50B780370FE
S3150800278070BC70470022030A8B420BD203098B42A6
S3150800279019D243088B422ED2411A00D20146524121
S315080027A010467047FF2209023FD012068B4205D316
S315080027B0121209028B4201D31212090203098B4233
S315080027C019D300E0090AC3098B4201D3CB01C01A09
S315080027D0524183098B4201D38B01C01A52414309E6
S315080027E08B4201D34B01C01A524103098B4201D3D4
S315080027F00B01C01A5241C3088B4201D3CB00C01A41
S31508002800524183088B4201D38B00C01A52414308B8
S315080028108B4201D34B00C01A5241884200D3401A5A
S315080028205241CFD201461046704708B500F088F8E5
S3150800283008BDFEE7F0B5020052B2002A23D50322EE
S315080028400F24374B05006DB22540083DAD08042618
S315080028507543060076B23440083CA408042674433F
S315080028601E59FF27BC461400044008277C436746C8
S31508002870A740BE438901C9B202400820424391409D
S31508002880314359511AE0274A0323040064B2A408C5
S3150800289004256C431459FF251E00064008277E436D
S315080028A0B540AC438901C9B2034008256B4399403A
S315080028B0214340B28008042358431150F0BD80B527
S315080028C0411E80225204914201D301200EE0401E8F
S315080028D01549086003210020C043FFF7ABFF00201D
S315080028E012490860072012490860002002BD80B519
S315080028F040B2FFF79FFF01BD80B5FFF7E0FF02BDBD
S3150800290000B5042805D10A48016804220A43026072
S3150800291004E00748016804229143016000BD0000F5
S315080029201CED00E000E400E014E000E018E000E040
S3150800293010E000E080B500F001F801BD7047FEE741
S315080029407047FEE710B50400002C01D1012037E0DE
S31508002950A0690028FFD16920205C002805D1002045
S3150800296068216054200000F08BFA24206921605405
S31508002970206800680121884321680860200000F06B
S31508002980B7F8012801D101201AE0606A002802D0B0
S31508002990200000F071F9206840680A490140206863
S315080029A04160206880682A218843216888602068F9
S315080029B000680121014320680160200000F0D0F979
S315080029C010BD0000FFB7FFFFFEB504001E0000277C
S315080029D038006A20205C202800D084E00D00002DF5
S315080029E005D06846028068460088002801D1012083
S315080029F07AE0A06880214901884207D12069002829
S31508002A0004D12800C00701D501206DE06820205CAC
S31508002A10012801D1022067E0012068216054E76699
S31508002A2022206A216054FFF77BFE029068460088E0
S31508002A3058216052684600885A216052A068802151
S31508002A40490188420AD12069002803D127485C2118
S31508002A50605210E0FF205C2160520CE0A06800285C
S31508002A6009D12069002803D1FF205C21605202E0C9
S31508002A707F205C2160525C20205A6946888007E0E6
S31508002A8028002168898C6A4692880A400280AD1C13
S31508002A905A20205A00281FD05A20205A401E5A2150
S31508002AA060520096029B00222021200000F098F92F
S31508002AB0002801D0032017E0A06880214901884238
S31508002AC002D120690028DBD02068808C6946898875
S31508002AD0014029706D1CDBE720206A2160546820BC
S31508002AE02754002000E00220FEBD0000FF01000080
S31508002AF0F8B504000021080010221000080008009C
S31508002B000D00A36826691E4367693743E3693B439B
S31508002B1026683668904F37403B43266833602368FB
S31508002B205B688E4E1E40E368334326687360A66969
S31508002B30236A33432668B668A54F37403B43266861
S31508002B40B3602368A34EB34214D1A34B1B689B07FB
S31508002B509B0F002B05D0022B08D005D3032B01D0E1
S31508002B6006E00CE002210AE0042108E0082106E05C
S31508002B70110004E02368994EB34200D01100802268
S31508002B801202E36993423CD1C9B2002906D0022950
S31508002B900FD0042915D008291ED026E0FFF79CFD82
S31508002BA0022148436168490840186168FFF7EAFD51
S31508002BB01CE060684008A44940186168FFF7E2FD18
S31508002BC014E0FFF74DFD02214843616849084018A3
S31508002BD06168FFF7D7FD09E060684008802149026F
S31508002BE040186168FFF7CEFD00E0012597490140CE
S31508002BF080B240084007400F084380B22168C86089
S31508002C0037E0C9B2002906D0022910D0042919D004
S31508002C10082923D02CE0FFF75FFD616849084018B2
S31508002C206168FFF7AFFD80B22168C86021E060687F
S31508002C304008874940186168FFF7A4FD80B22168FB
S31508002C40C86016E0FFF70CFD61684908401861681E
S31508002C50FFF798FD80B22168C8600AE060684008FE
S31508002C6080186168FFF78EFD80B22168C86000E0B1
S31508002C7001252800C0B2F2BD00B52421415CC90770
S31508002C8007D501684968734A0A40816A1143026890
S31508002C9051602421415C890707D5016849686E4A55
S31508002CA00A40C16A1143026851602421415C490700
S31508002CB007D501684968694A0A40016B11430268E9
S31508002CC051602421415C090707D501684968644AAF
S31508002CD00A40416B1143026851602421415CC906D0
S31508002CE007D5016889685F4A0A40816B1143026803
S31508002CF091602421415C890607D5016889685A4A8A
S31508002D000A40C16B1143026891602421415C49065F
S31508002D1014D501684968554A0A40016C114302688E
S31508002D205160016C80225203914207D101684968BB
S31508002D304F4A0A40416C1143026851602421415CA4
S31508002D40090607D5016849684A4A0A40816C114351
S31508002D500068416000BD0000F369FFFFFFCFFFFF79
S31508002D607CB5040000252800E566FFF7D9FC0600B7
S31508002D7020681849884221D12068006800070CD5C8
S31508002D803D4800903300002280218903200000F08E
S31508002D9027F8002801D0032018E0206800684007BB
S31508002DA00CD535480090330000228021C903200045
S31508002DB000F016F8002801D0032007E0202069213A
S31508002DC060546A21605468202554002076BD0000AE
S31508002DD0FFF4FFFF00380140301002400044004075
S31508002DE0F4B504000D001F00069E2068C06928403F
S31508002DF0A84201D1012000E00020694609788842EE
S31508002E0020D10020C0438642EFD0002E04D0FFF721
S31508002E1087FCC01B8642E8D2206800681749014033
S31508002E2020680160206880680121884321688860DD
S31508002E302020692160546A2160540020682160546A
S31508002E40032000E00020F2BD0024F400F0FF00009B
S31508002E5000127A00FFFFFDFFFFFFFEFFFFFFFBFFEB
S31508002E60FF7FFFFFFFEFFFFFFFDFFFFFFFFFEFFF24
S31508002E70FFFF9FFFFFFFF7FFFFFFFF015FFEFFFF5B
S31508002E807047FEE7F8B5020000230020002032E074
S31508002E90052403E0724CA242FAD134001F003E40DA
S31508002EA004277E43B44004436E489E0804277E43A5
S31508002EB084516D4C2068A8434E68F60300D5284314
S31508002EC020606A4C2068A8434E68B60300D528439C
S31508002ED02060674C2068A8434E68F60200D5284350
S31508002EE02060644C2068A8434E68B60201D50543A5
S31508002EF0280020605B1C0868D840002800D1AEE096
S31508002F000124086825009D400540002DF2D0486838
S31508002F10022802D0486812281ED1D8080426704311
S31508002F201018076A072000970F26B4461F000740A7
S31508002F30042677436646BE40009FB743BC460E69E3
S31508002F401F00384004277843864067463E43D80822
S31508002F50042778431018066217680326BC461F0024
S31508002F60022047433000B8406746874300974868C1
S31508002F70304084461F00022047436046B840009F01
S31508002F80384310604868012808D04868022805D0E8
S31508002F904868112802D0486812281DD19768BC468F
S31508002FA01F00022047433000B84067468743009712
S31508002FB0C86884461F00022047436046B840009F01
S31508002FC0384390605768200098408743486800094E
S31508002FD02040984038435060D768BC461F000220FE
S31508002FE047433000B8406746874300978868844659
S31508002FF01F00022047436046B840009F3843D06010
S315080030004868C00000D475E720480768274307606A
S315080030100068204000900098124884469F080420C3
S3150800302047436046C05900900F27BC461F00300032
S31508003030384004277843674687400098B843902766
S31508003040FF05BA4201D1002428E7114FBA4200D140
S3150800305024E7104CA24200D01CE702241EE7F1BD6B
S31508003060000C004808000140000401400404014027
S31508003070080401400C04014000B5D2B2002A02D06F
S3150800308089B2816101E089B2816200BD18100240EF
S31508003090000400480008004880B500F007F800F072
S315080030A097F800F01BF900F097F8FAE780B500F0FA
S315080030B03DF900F005F800F009F900F047F901BDFF
S315080030C038B590B0012004900520059002240C9490
S315080030D0802040020D90802040030E9000250F9519
S315080030E004A8FEF7EFFF002800D0FEE707200090AF
S315080030F001940295039501216846FFF7FDF900281A
S3150800310000D0FEE711B030BD38B586B00124274897
S3150800311001682143016000682040009000988020E3
S31508003120800223490A6802430A600A68024000923C
S31508003130009A802212030B6813430B6009680A4041
S31508003140009200991B490A6802430A600968084008
S3150800315000900098002200210420C043FFF7C7FB17
S31508003160002200210120C043FFF7C1FB00220021F5
S315080031700020C043FFF7BBFB80208000019002942B
S3150800318000250395049501A90B48FFF77BFE0C2043
S31508003190019002200290039503200490059401A94A
S315080031A09020C005FFF76EFE07B030BD181002402C
S315080031B0141002401C1002400008004800B5BFF376
S315080031C04F8F3A483A490860BFF34F8F00BFFDE773
S315080031D080B500F009F801BD80B500F019F801BD09
S315080031E080B5FFF7EBFF01BD80B532483249016073
S315080031F0E1210902416000218160C16001610C2260
S3150800320042618161C16101624162FFF79BFB01BDB9
S3150800321070B52A4C2078002815D1294D280000F0D1
S3150800322037F8012833D12878002830D02878412863
S315080032302DDA00F09EF8234908600120207000204E
S315080032402149087023E0204D1D4E28783018401C6F
S3150800325000F01EF8012811D12878401C287028781B
S315080032603178884213D1002020707078FF280ED15B
S31508003270287802280BD1FFF7B3FF08E000F079F8A9
S31508003280104909686431814201D20020207070BD5E
S3150800329080B50100002301220648FFF795FBC0B25E
S315080032A0002801D1012000E0002002BD0400FA0533
S315080032B00CED00E0C4000020004400408501002019
S315080032C034010020780100208401002080B5002206
S315080032D0802189001248FFF7CFFE01BD38B500F0FE
S315080032E048F804000F4D2868201AFA214900884238
S315080032F015D30D480178002908D101210170012252
S31508003300802189000648FFF7B7FE07E00021017013
S315080033100022802189000248FFF7AEFE2C6031BDED
S31508003320000800487C0100208601002080B5064878
S31508003330016810220A4302600020FFF7F7F9FFF739
S31508003340E3FE002002BD00000020024080B5FFF722
S31508003350BDF9FA218900FFF715FAFFF7CDFA04201F
S31508003360FFF7CEFA002200210020C043FFF7BFFA7C
S3150800337001BD80B5FFF7D4F902BD80B500F004F8A9
S31508003380FFF7D8FA01BDFEE702480168491C01604B
S31508003390704700BF800100201448016801220A43D3
S315080033A0026013490A68134B13400B600268124BFC
S315080033B0134003600268114B134003600868104A03
S315080033C002400A600F4801680F22914301600E48C7
S315080033D001680E4A0A4002600D48016801229143BD
S315080033E0016000200B490860704700000010024089
S315080033F0041002400CB8FFF8FFFFF6FEFFFFFBFFC4
S31508003400FFFFC0FF2C10024030100240ACFEFFFF49
S31508003410341002400810024070B40123002413E05F
S315080034200168001D194202D04D466D1E49190C60EF
S31508003430091D121F042AFAD20D00960701D50C8021
S31508003440AD1C1A4000D02C700268001D002AE7D176
S3150800345070BC704730B401220EE00368C318446894
S315080034600830144202D04D466D1E64191D68256049
S315080034701B1D241D091FF9D10168001D0029ECD167
S3150800348030BC704710B5074979441831064C7C445E
S31508003490163404E0081D0A68891888470100A14205
S315080034A0F8D110BD08000000280000006DFFFFFFDE
S315080034B0C4000000C40000200000000099FFFFFFC0
S315080034C004000000B4000000C00000200000000056
S315080034D000F00DF8002801D0FFF7D4FF00BF00BFA9
S315080034E0002000BF00BFFFF7D7FD00F002F801205B
S315080034F0704780B500F002F801BDFEE7074638467A
S3150800350000F002F8FBE7FEE780B500BF00BF024AFD
S3150800351011001820ABBEFBE72600020002488546CC
S31508003520024880470248004788050020993300086A
S315080035306535000802030405060708090A0B0C0D81
S315080035400E0F10100102030405060708090A0B0CE2
S315080035500D0E0F1000000000000000000102030419
S315080035600607080900BF00BF00BF00BFFFF7B0FF8E
S31508003570000000000102030400127A00FEE7FEE7DD
S31508003580FEE7FEE7FEE7FEE7FEE7FEE7FEE7FEE705
S31508003590FEE7FEE7FEE7FEE7FEE7FEE7FEE7FEE7F5
S315080035A0FEE7FEE7FEE7FEE7FEE7FEE7FEE7FEE7E5
S7050800356558
